LX51 LINKER/LOCATER V4.17                                                               06/13/2011  13:18:25  PAGE 1


LX51 LINKER/LOCATER V4.17, INVOKED BY:
C:\KEIL\C51\BIN\LX51.EXE STARTUP.obj, Main.obj TO nRF24LE1 CLASSES (XDATA (X:0X0-X:0X3FF, X:0XFA00-X:0XFFFF), HDATA (X:0
>> X0-X:0X3FF, X:0XFA00-X:0XFFFF), CODE (C:0X0-C:0X3FFF), CONST (C:0X0-C:0X3FFF), ECODE (C:0X0-C:0X3FFF), HCONST (C:0X0-
>> C:0X3FFF))


CPU MODE:     8051 MODE
MEMORY MODEL: COMPACT


INPUT MODULES INCLUDED:
  STARTUP.obj (?C_STARTUP)
         COMMENT TYPE 0: AX51 V3.03
  Main.obj (MAIN)
         COMMENT TYPE 0: C51 V8.09
  C:\KEIL\C51\LIB\C51C.LIB (?C_INIT)
         COMMENT TYPE 1: A51 / ASM51 Assembler
  C:\KEIL\C51\LIB\C51C.LIB (?C?CLDPTR)
         COMMENT TYPE 1: A51 / ASM51 Assembler


ACTIVE MEMORY CLASSES OF MODULE:  nRF24LE1 (?C_STARTUP)

BASE        START       END         USED      MEMORY CLASS
==========================================================
X:000000H   X:000000H   X:0003FFH             XDATA
            X:00FA00H   X:00FFFFH               
X:000000H   X:000000H   X:0003FFH             HDATA
            X:00FA00H   X:00FFFFH               
C:000000H   C:000000H   C:003FFFH   0002B0H   CODE
C:000000H   C:000000H   C:003FFFH             CONST
C:000000H   C:000000H   C:003FFFH             ECODE
B00:0000H   C:000000H   C:003FFFH             HCONST
I:000000H   I:000000H   I:0000FFH   000001H   IDATA
X:000000H   X:000000H   X:0000FFH   00000BH   PDATA
I:000000H   I:000000H   I:00007FH   000013H   DATA


MEMORY MAP OF MODULE:  nRF24LE1 (?C_STARTUP)


START     STOP      LENGTH    ALIGN  RELOC    MEMORY CLASS   SEGMENT NAME
=========================================================================

* * * * * * * * * * *   D A T A   M E M O R Y   * * * * * * * * * * * * *
000000H   000007H   000008H   ---    AT..     DATA           "REG BANK 0"
000008H   000011H   00000AH   BYTE   UNIT     DATA           ?DT?MAIN
000012H   00001FH   00000EH   ---    ---      **GAP**
000020H   000020H   000001H   BYTE   BITADDR  DATA           ?BA?MAIN
000021H   000021H   000001H   BYTE   UNIT     IDATA          ?STACK

* * * * * * * * * * *   C O D E   M E M O R Y   * * * * * * * * * * * * *
000000H   000002H   000003H   ---    OFFS..   CODE           ?CO?STARTUP?3
000003H   00000AH   000008H   BYTE   UNIT     CODE           ?PR?ADC_START?MAIN
00000BH   00000DH   000003H   BYTE   OFFS..   CODE           ?MAIN?0000B
00000EH   000049H   00003CH   BYTE   UNIT     CODE           ?PR?_SPI_WRITE_BUF?MAIN
00004AH   00004AH   000001H   ---    ---      **GAP**
00004BH   00004DH   000003H   BYTE   OFFS..   CODE           ?MAIN?0004B
00004EH   000067H   00001AH   BYTE   UNIT     CODE           ?PR?IO_INIT?MAIN
000068H   00006AH   000003H   BYTE   UNIT     CODE           ?PR?RTC2_IRQ?MAIN
00006BH   00006DH   000003H   BYTE   OFFS..   CODE           ?MAIN?0006B
00006EH   0000F9H   00008CH   BYTE   UNIT     CODE           ?C_C51STARTUP
0000FAH   00014EH   000055H   BYTE   UNIT     CODE           ?PR?RF_INIT?MAIN
00014FH   000188H   00003AH   BYTE   UNIT     CODE           ?PR?TX_MODE?MAIN
000189H   0001BDH   000035H   BYTE   UNIT     CODE           ?PR?MAIN?MAIN
0001BEH   0001E9H   00002CH   BYTE   UNIT     CODE           ?PR?_DELAY?MAIN
LX51 LINKER/LOCATER V4.17                                                             06/13/2011  13:18:25  PAGE 2


0001EAH   00020FH   000026H   BYTE   UNIT     CODE           ?PR?RF_IRQ?MAIN
000210H   000228H   000019H   BYTE   UNIT     CODE           ?C?LIB_CODE
000229H   00023CH   000014H   BYTE   UNIT     CODE           ?C_INITSEG
00023DH   00024DH   000011H   BYTE   UNIT     CODE           ?PR?_SPI_RW_REG?MAIN
00024EH   00025CH   00000FH   BYTE   UNIT     CODE           ?PR?RTC2_INIT?MAIN
00025DH   000269H   00000DH   BYTE   UNIT     CODE           ?PR?_SPI_READ?MAIN
00026AH   000276H   00000DH   BYTE   UNIT     CODE           ?PR?RTC0_INIT?MAIN
000277H   000283H   00000DH   BYTE   UNIT     CODE           ?PR?RTC0_IRQ?MAIN
000284H   00028DH   00000AH   BYTE   UNIT     CODE           ?PR?_SPI_RW?MAIN
00028EH   000297H   00000AH   BYTE   UNIT     CODE           ?PR?ADC_INIT?MAIN
000298H   0002A0H   000009H   BYTE   UNIT     CODE           ?PR?PD_MODE?MAIN
0002A1H   0002A8H   000008H   BYTE   UNIT     CODE           ?PR?GET_ADC_VALUE?MAIN
0002A9H   0002ACH   000004H   BYTE   UNIT     CODE           ?PR?RTC2_ON?MAIN
0002ADH   0002B0H   000004H   BYTE   UNIT     CODE           ?PR?RTC2_OFF?MAIN

* * * * * * * * * * *  X D A T A   M E M O R Y  * * * * * * * * * * * * *
000000H   000005H   000006H   BYTE   INPAGE   PDATA          _PDATA_GROUP_
000006H   00000AH   000005H   BYTE   INPAGE   PDATA          ?PD?MAIN



OVERLAY MAP OF MODULE:   nRF24LE1 (?C_STARTUP)


FUNCTION/MODULE             PDATA_GROUP
--> CALLED FUNCTION/MODULE  START  STOP
=======================================
?C_C51STARTUP               ----- -----
  +--> ?PR?MAIN?MAIN
  +--> ?C_INITSEG

MAIN/MAIN                   0000H 0000H
  +--> ?PR?IO_INIT?MAIN
  +--> ?PR?RF_INIT?MAIN
  +--> ?PR?ADC_INIT?MAIN
  +--> ?PR?ADC_START?MAIN
  +--> ?PR?GET_ADC_VALUE?MAIN
  +--> ?PR?TX_MODE?MAIN
  +--> ?PR?_DELAY?MAIN

IO_INIT/MAIN                ----- -----
  +--> ?PR?_DELAY?MAIN

_DELAY/MAIN                 0001H 0002H

RF_INIT/MAIN                ----- -----
  +--> ?PR?_DELAY?MAIN
  +--> ?PR?_SPI_WRITE_BUF?MAIN
  +--> ?PR?_SPI_RW_REG?MAIN

_SPI_WRITE_BUF/MAIN         0001H 0005H
  +--> ?PR?_SPI_RW?MAIN

_SPI_RW/MAIN                ----- -----

_SPI_RW_REG/MAIN            ----- -----
  +--> ?PR?_SPI_RW?MAIN

ADC_INIT/MAIN               ----- -----

ADC_START/MAIN              ----- -----

GET_ADC_VALUE/MAIN          ----- -----

TX_MODE/MAIN                ----- -----
LX51 LINKER/LOCATER V4.17                                                             06/13/2011  13:18:25  PAGE 3


  +--> ?PR?_SPI_RW_REG?MAIN
  +--> ?PR?_SPI_WRITE_BUF?MAIN
  +--> ?PR?_DELAY?MAIN

?C_INITSEG                  ----- -----

*** NEW ROOT **************

RF_IRQ/MAIN                 ----- -----
  +--> ?PR?_SPI_READ?MAIN
  +--> ?PR?_SPI_RW_REG?MAIN

_SPI_READ/MAIN              ----- -----
  +--> ?PR?_SPI_RW?MAIN

*** NEW ROOT **************

RTC2_IRQ/MAIN               ----- -----

*** NEW ROOT **************

RTC0_IRQ/MAIN               ----- -----



PUBLIC SYMBOLS OF MODULE:  nRF24LE1 (?C_STARTUP)


      VALUE       CLASS    TYPE      PUBLIC SYMBOL NAME
      =================================================
      02000001H   PDATA    BYTE      ?_SPI_Write_Buf?BYTE
      01000210H   CODE     ---       ?C?CLDPTR
      00000000H   NUMBER   ---       ?C?CODESEG
      00000000H   NUMBER   ---       ?C?XDATASEG
      010000B5H   CODE     ---       ?C_START
      01000000H   CODE     NEAR LAB  ?C_STARTUP
      010001BEH   CODE     ---       _delay
      0100025DH   CODE     ---       _SPI_Read
      01000284H   CODE     ---       _SPI_RW
      0100023DH   CODE     ---       _SPI_RW_Reg
      0100000EH   CODE     ---       _SPI_Write_Buf
*SFR* 000000D0H.6 DATA     BIT       AC
*SFR* 000000E0H   DATA     BYTE      ACC
      0100028EH   CODE     ---       adc_init
      01000003H   CODE     ---       adc_start
*SFR* 000000D3H   DATA     BYTE      ADCCON1
*SFR* 000000D2H   DATA     BYTE      ADCCON2
*SFR* 000000D1H   DATA     BYTE      ADCCON3
*SFR* 000000D4H   DATA     BYTE      ADCDATH
*SFR* 000000D5H   DATA     BYTE      ADCDATL
*SFR* 000000D8H   DATA     BYTE      ADCON
*SFR* 000000EFH   DATA     BYTE      ARCON
*SFR* 000000F0H   DATA     BYTE      B
*SFR* 000000D8H.7 DATA     BIT       BD
*SFR* 000000C2H   DATA     WORD      CC1
*SFR* 000000C4H   DATA     WORD      CC2
*SFR* 000000C6H   DATA     WORD      CC3
*SFR* 000000C1H   DATA     BYTE      CCEN
*SFR* 000000C3H   DATA     BYTE      CCH1
*SFR* 000000C5H   DATA     BYTE      CCH2
*SFR* 000000C7H   DATA     BYTE      CCH3
*SFR* 000000C2H   DATA     BYTE      CCL1
*SFR* 000000C4H   DATA     BYTE      CCL2
*SFR* 000000C6H   DATA     BYTE      CCL3
*SFR* 000000DDH   DATA     BYTE      CCPDATIA
LX51 LINKER/LOCATER V4.17                                                             06/13/2011  13:18:25  PAGE 4


*SFR* 000000DEH   DATA     BYTE      CCPDATIB
*SFR* 000000DFH   DATA     BYTE      CCPDATO
*SFR* 000000A3H   DATA     BYTE      CLKCTRL
*SFR* 000000ADH   DATA     BYTE      CLKLFCTRL
*SFR* 000000DBH   DATA     BYTE      COMPCON
*SFR* 000000CAH   DATA     WORD      CRC
*SFR* 000000CBH   DATA     BYTE      CRCH
*SFR* 000000CAH   DATA     BYTE      CRCL
*SFR* 000000D0H.7 DATA     BIT       CY
*SFR* 00000083H   DATA     BYTE      DPH
*SFR* 00000085H   DATA     BYTE      DPH1
*SFR* 00000082H   DATA     BYTE      DPL
*SFR* 00000084H   DATA     BYTE      DPL1
*SFR* 00000092H   DATA     BYTE      DPS
*SFR* 000000A8H.7 DATA     BIT       EA
*SFR* 000000A8H.4 DATA     BIT       ES0
*SFR* 000000A8H.1 DATA     BIT       ET0
*SFR* 000000A8H.3 DATA     BIT       ET1
*SFR* 000000A8H.5 DATA     BIT       ET2
*SFR* 000000A8H   DATA     BIT       EX0
*SFR* 000000A8H.2 DATA     BIT       EX1
*SFR* 000000B8H.7 DATA     BIT       EXEN2
*SFR* 000000C0H.7 DATA     BIT       EXF2
*SFR* 000000D0H.5 DATA     BIT       F0
*SFR* 000000FAH   DATA     BYTE      FCR
*SFR* 000000FBH   DATA     BYTE      FDCR
*SFR* 000000F9H   DATA     BYTE      FPCR
*SFR* 000000F8H   DATA     BYTE      FSR
      010002A1H   CODE     ---       get_adc_value
*SFR* 000000C8H.5 DATA     BIT       I2FR
*SFR* 000000C8H.6 DATA     BIT       I3FR
      00000008H   DATA     ---       id_buf
*SFR* 00000088H.1 DATA     BIT       IE0
*SFR* 00000088H.3 DATA     BIT       IE1
*SFR* 000000A8H   DATA     BYTE      IEN0
*SFR* 000000B8H   DATA     BYTE      IEN1
*SFR* 000000F8H.3 DATA     BIT       INFEN
*SFR* 000000A6H   DATA     BYTE      INTEXP
      0100004EH   CODE     ---       io_init
*SFR* 000000A9H   DATA     BYTE      IP0
*SFR* 000000B9H   DATA     BYTE      IP1
*SFR* 000000C0H   DATA     BYTE      IRCON
*SFR* 00000088H   DATA     BIT       IT0
*SFR* 00000088H.2 DATA     BIT       IT1
*SFR* 00000080H   DATA     BIT       LED1
*SFR* 00000080H.5 DATA     BIT       LED2
*SFR* 00000080H.1 DATA     BIT       LED3
      01000189H   CODE     ---       main
      00000020H.4 DATA     BIT       MAX_RT
*SFR* 000000F8H.7 DATA     BIT       MCDIS
*SFR* 000000E9H   DATA     BYTE      MD0
*SFR* 000000EAH   DATA     BYTE      MD1
*SFR* 000000EBH   DATA     BYTE      MD2
*SFR* 000000ECH   DATA     BYTE      MD3
*SFR* 000000EDH   DATA     BYTE      MD4
*SFR* 000000EEH   DATA     BYTE      MD5
*SFR* 000000A7H   DATA     BYTE      MEMCON
*SFR* 000000B8H.4 DATA     BIT       MISC
*SFR* 000000C0H.4 DATA     BIT       MISCF
*SFR* 000000C9H   DATA     BYTE      MPAGE
*SFR* 000000AEH   DATA     BYTE      OPMCON
*SFR* 000000D0H.2 DATA     BIT       OV
*SFR* 000000D0H   DATA     BIT       P
*SFR* 00000080H   DATA     BYTE      P0
*SFR* 00000080H   DATA     BIT       P00
LX51 LINKER/LOCATER V4.17                                                             06/13/2011  13:18:25  PAGE 5


*SFR* 00000080H.1 DATA     BIT       P01
*SFR* 00000080H.2 DATA     BIT       P02
*SFR* 00000080H.3 DATA     BIT       P03
*SFR* 00000080H.4 DATA     BIT       P04
*SFR* 00000080H.5 DATA     BIT       P05
*SFR* 00000080H.6 DATA     BIT       P06
*SFR* 00000080H.7 DATA     BIT       P07
*SFR* 0000009EH   DATA     BYTE      P0CON
*SFR* 00000093H   DATA     BYTE      P0DIR
*SFR* 00000090H   DATA     BYTE      P1
*SFR* 00000090H   DATA     BIT       P10
*SFR* 00000090H.1 DATA     BIT       P11
*SFR* 00000090H.2 DATA     BIT       P12
*SFR* 00000090H.3 DATA     BIT       P13
*SFR* 00000090H.4 DATA     BIT       P14
*SFR* 00000090H.5 DATA     BIT       P15
*SFR* 00000090H.6 DATA     BIT       P16
*SFR* 00000090H.7 DATA     BIT       P17
*SFR* 0000009FH   DATA     BYTE      P1CON
*SFR* 00000094H   DATA     BYTE      P1DIR
*SFR* 000000A0H   DATA     BYTE      P2
*SFR* 000000A0H   DATA     BIT       P20
*SFR* 000000A0H.1 DATA     BIT       P21
*SFR* 000000A0H.2 DATA     BIT       P22
*SFR* 000000A0H.3 DATA     BIT       P23
*SFR* 000000A0H.4 DATA     BIT       P24
*SFR* 000000A0H.5 DATA     BIT       P25
*SFR* 000000A0H.6 DATA     BIT       P26
*SFR* 000000A0H.7 DATA     BIT       P27
*SFR* 00000097H   DATA     BYTE      P2CON
*SFR* 00000095H   DATA     BYTE      P2DIR
*SFR* 000000B0H   DATA     BYTE      P3
*SFR* 000000B0H   DATA     BIT       P30
*SFR* 000000B0H.1 DATA     BIT       P31
*SFR* 000000B0H.2 DATA     BIT       P32
*SFR* 000000B0H.3 DATA     BIT       P33
*SFR* 000000B0H.4 DATA     BIT       P34
*SFR* 000000B0H.5 DATA     BIT       P35
*SFR* 000000B0H.6 DATA     BIT       P36
*SFR* 000000B0H.7 DATA     BIT       P37
*SFR* 0000008FH   DATA     BYTE      P3CON
*SFR* 00000096H   DATA     BYTE      P3DIR
*SFR* 00000087H   DATA     BYTE      PCON
      01000298H   CODE     ---       PD_Mode
*SFR* 000000DCH   DATA     BYTE      POFCON
*SFR* 000000A0H   DATA     BYTE      PPAGE_SFR
*SFR* 000000D0H   DATA     BYTE      PSW
*SFR* 000000B2H   DATA     BYTE      PWMCON
*SFR* 000000A1H   DATA     BYTE      PWMDC0
*SFR* 000000A2H   DATA     BYTE      PWMDC1
*SFR* 000000A4H   DATA     BYTE      PWRDWN
*SFR* 00000098H.2 DATA     BIT       RB80
*SFR* 000000F8H.1 DATA     BIT       RDEND
*SFR* 000000F8H.2 DATA     BIT       RDIS
*SFR* 000000F8H.4 DATA     BIT       RDYN
*SFR* 00000098H.4 DATA     BIT       REN0
*SFR* 000000B8H.1 DATA     BIT       RF
      010000FAH   CODE     ---       rf_init
      010001EAH   CODE     ---       RF_IRQ
*SFR* 000000E8H   DATA     BIT       RFCE
*SFR* 000000E8H.2 DATA     BIT       RFCKEN
*SFR* 000000E8H   DATA     BYTE      RFCON
*SFR* 000000E8H.1 DATA     BIT       RFCSN
*SFR* 000000C0H.1 DATA     BIT       RFF
*SFR* 000000B8H   DATA     BIT       RFSPI
LX51 LINKER/LOCATER V4.17                                                             06/13/2011  13:18:25  PAGE 6


*SFR* 000000C0H   DATA     BIT       RFSPIF
*SFR* 00000098H   DATA     BIT       RI0
*SFR* 000000D6H   DATA     BYTE      RNGCTL
*SFR* 000000D7H   DATA     BYTE      RNGDAT
*SFR* 000000D0H.3 DATA     BIT       RS0
*SFR* 000000D0H.4 DATA     BIT       RS1
*SFR* 000000B1H   DATA     BYTE      RSTREAS
      0100026AH   CODE     ---       rtc0_init
      01000277H   CODE     ---       RTC0_IRQ
      0100024EH   CODE     ---       rtc2_init
      01000068H   CODE     ---       RTC2_IRQ
      010002ADH   CODE     ---       rtc2_off
      010002A9H   CODE     ---       rtc2_on
*SFR* 000000B4H   DATA     BYTE      RTC2CMP0
*SFR* 000000B5H   DATA     BYTE      RTC2CMP1
*SFR* 000000B3H   DATA     BYTE      RTC2CON
*SFR* 000000B6H   DATA     BYTE      RTC2CPT00
*SFR* 000000ABH   DATA     BYTE      RTC2CPT01
*SFR* 000000ACH   DATA     BYTE      RTC2CPT10
      00000020H.6 DATA     BIT       RX_DR
*SFR* 00000099H   DATA     BYTE      S0BUF
*SFR* 00000098H   DATA     BYTE      S0CON
*SFR* 000000BAH   DATA     BYTE      S0RELH
*SFR* 000000AAH   DATA     BYTE      S0RELL
*SFR* 00000090H.2 DATA     BIT       S1
*SFR* 00000090H.3 DATA     BIT       S2
*SFR* 00000090H.4 DATA     BIT       S3
*SFR* 00000098H.7 DATA     BIT       SM0
*SFR* 00000098H.6 DATA     BIT       SM1
*SFR* 00000098H.5 DATA     BIT       SM20
*SFR* 00000081H   DATA     BYTE      SP
*SFR* 000000B8H.2 DATA     BIT       SPI
*SFR* 000000C0H.2 DATA     BIT       SPIF
*SFR* 000000FCH   DATA     BYTE      SPIMCON0
*SFR* 000000FDH   DATA     BYTE      SPIMCON1
*SFR* 000000FFH   DATA     BYTE      SPIMDAT
*SFR* 000000FEH   DATA     BYTE      SPIMSTAT
*SFR* 000000E4H   DATA     BYTE      SPIRCON0
*SFR* 000000E5H   DATA     BYTE      SPIRCON1
*SFR* 000000E7H   DATA     BYTE      SPIRDAT
*SFR* 000000E6H   DATA     BYTE      SPIRSTAT
*SFR* 000000BCH   DATA     BYTE      SPISCON0
*SFR* 000000BDH   DATA     BYTE      SPISCON1
*SFR* 000000BFH   DATA     BYTE      SPISDAT
*SFR* 000000B7H   DATA     BYTE      SPISRDSZ
*SFR* 000000BEH   DATA     BYTE      SPISSTAT
      00000020H   DATA     BYTE      sta
*SFR* 000000F8H.6 DATA     BIT       STP
*SFR* 000000CCH   DATA     WORD      T2
*SFR* 000000C8H.2 DATA     BIT       T2CM
*SFR* 000000C8H   DATA     BYTE      T2CON
*SFR* 000000C8H   DATA     BIT       T2I0
*SFR* 000000C8H.1 DATA     BIT       T2I1
*SFR* 000000C8H.7 DATA     BIT       T2PS
*SFR* 000000C8H.3 DATA     BIT       T2R0
*SFR* 000000C8H.4 DATA     BIT       T2R1
*SFR* 00000098H.3 DATA     BIT       TB80
*SFR* 00000088H   DATA     BYTE      TCON
*SFR* 00000088H.5 DATA     BIT       TF0
*SFR* 00000088H.7 DATA     BIT       TF1
*SFR* 000000C0H.6 DATA     BIT       TF2
*SFR* 0000008CH   DATA     BYTE      TH0
*SFR* 0000008DH   DATA     BYTE      TH1
*SFR* 000000CDH   DATA     BYTE      TH2
*SFR* 00000098H.1 DATA     BIT       TI0
LX51 LINKER/LOCATER V4.17                                                             06/13/2011  13:18:25  PAGE 7


*SFR* 0000008AH   DATA     BYTE      TL0
*SFR* 0000008BH   DATA     BYTE      TL1
*SFR* 000000CCH   DATA     BYTE      TL2
*SFR* 00000089H   DATA     BYTE      TMOD
*SFR* 00000088H.4 DATA     BIT       TR0
*SFR* 00000088H.6 DATA     BIT       TR1
      02000006H   PDATA    ---       TX_ADDRESS
      00000020H.5 DATA     BIT       TX_DS
      0100014FH   CODE     ---       TX_Mode
*SFR* 000000E2H   DATA     BYTE      W2CON0
*SFR* 000000E1H   DATA     BYTE      W2CON1
*SFR* 000000DAH   DATA     BYTE      W2DAT
*SFR* 000000D9H   DATA     BYTE      W2SADR
*SFR* 000000AFH   DATA     BYTE      WDSV
*SFR* 000000F8H.5 DATA     BIT       WEN
*SFR* 000000F8H   DATA     BIT       WPEN
*SFR* 000000A5H   DATA     BYTE      WUCON
*SFR* 000000C0H.5 DATA     BIT       WUF
*SFR* 000000B8H.5 DATA     BIT       WUIRQ
*SFR* 000000CFH   DATA     BYTE      WUOPC0
*SFR* 000000CEH   DATA     BYTE      WUOPC1
*SFR* 000000B8H.3 DATA     BIT       WUPIN
*SFR* 000000C0H.3 DATA     BIT       WUPINF



SYMBOL TABLE OF MODULE:  nRF24LE1 (?C_STARTUP)

      VALUE       REP       CLASS    TYPE      SYMBOL NAME
      ====================================================
      ---         MODULE    ---      ---       ?C_STARTUP
      01000000H   PUBLIC    CODE     NEAR LAB  ?C_STARTUP
      000000E0H   SFRSYM    DATA     BYTE      ACC
      000000F0H   SFRSYM    DATA     BYTE      B
      00000083H   SFRSYM    DATA     BYTE      DPH
      00000082H   SFRSYM    DATA     BYTE      DPL
      000000A0H   SFRSYM    DATA     BYTE      PPAGE_SFR
      00000081H   SFRSYM    DATA     BYTE      SP
      00000000H   SYMBOL    NUMBER   ---       IBPSTACK
      00000100H   SYMBOL    NUMBER   ---       IBPSTACKTOP
      00000080H   SYMBOL    NUMBER   ---       IDATALEN
      01000071H   SYMBOL    CODE     NEAR LAB  IDATALOOP
      00000000H   SYMBOL    NUMBER   ---       PBPSTACK
      00010000H   SYMBOL    NUMBER   ---       PBPSTACKTOP
      00000000H   SYMBOL    NUMBER   ---       PDATALEN
      00000000H   SYMBOL    NUMBER   ---       PDATASTART
      00000000H   SYMBOL    NUMBER   ---       PPAGE
      00000000H   SYMBOL    NUMBER   ---       PPAGEENABLE
      0100006EH   SYMBOL    CODE     NEAR LAB  STARTUP1
      00000000H   SYMBOL    NUMBER   ---       XBPSTACK
      00010000H   SYMBOL    NUMBER   ---       XBPSTACKTOP
      00000000H   SYMBOL    NUMBER   ---       XDATALEN
      00000000H   SYMBOL    NUMBER   ---       XDATASTART

      01000000H   BLOCK     CODE     NEAR LAB  LVL=0
      01000000H   LINE      CODE     ---       #92
      ---         BLOCKEND  ---      ---       LVL=0

      0100006EH   BLOCK     CODE     NEAR LAB  LVL=0
      0100006EH   LINE      CODE     ---       #99
      01000070H   LINE      CODE     ---       #100
      01000071H   LINE      CODE     ---       #101
      01000072H   LINE      CODE     ---       #102
      01000074H   LINE      CODE     ---       #151
      01000077H   LINE      CODE     ---       #155
LX51 LINKER/LOCATER V4.17                                                             06/13/2011  13:18:25  PAGE 8


      ---         BLOCKEND  ---      ---       LVL=0

      ---         MODULE    ---      ---       MAIN
      00000020H.4 PUBLIC    DATA     BIT       MAX_RT
      00000008H   PUBLIC    DATA     ---       id_buf
      00000020H.5 PUBLIC    DATA     BIT       TX_DS
      00000020H.6 PUBLIC    DATA     BIT       RX_DR
      00000020H   PUBLIC    DATA     BYTE      sta
      02000006H   PUBLIC    PDATA    ---       TX_ADDRESS
      01000189H   PUBLIC    CODE     ---       main
      010002A1H   PUBLIC    CODE     ---       get_adc_value
      01000003H   PUBLIC    CODE     ---       adc_start
      0100028EH   PUBLIC    CODE     ---       adc_init
      0100004EH   PUBLIC    CODE     ---       io_init
      01000277H   PUBLIC    CODE     ---       RTC0_IRQ
      01000068H   PUBLIC    CODE     ---       RTC2_IRQ
      010002ADH   PUBLIC    CODE     ---       rtc2_off
      010002A9H   PUBLIC    CODE     ---       rtc2_on
      0100026AH   PUBLIC    CODE     ---       rtc0_init
      0100024EH   PUBLIC    CODE     ---       rtc2_init
      010001EAH   PUBLIC    CODE     ---       RF_IRQ
      010000FAH   PUBLIC    CODE     ---       rf_init
      0100014FH   PUBLIC    CODE     ---       TX_Mode
      01000298H   PUBLIC    CODE     ---       PD_Mode
      02000001H   PUBLIC    PDATA    BYTE      ?_SPI_Write_Buf?BYTE
      0100000EH   PUBLIC    CODE     ---       _SPI_Write_Buf
      0100025DH   PUBLIC    CODE     ---       _SPI_Read
      0100023DH   PUBLIC    CODE     ---       _SPI_RW_Reg
      01000284H   PUBLIC    CODE     ---       _SPI_RW
      010001BEH   PUBLIC    CODE     ---       _delay
      00000098H.3 SFRSYM    DATA     BIT       TB80
      000000BEH   SFRSYM    DATA     BYTE      SPISSTAT
      000000C8H   SFRSYM    DATA     BIT       T2I0
      000000C3H   SFRSYM    DATA     BYTE      CCH1
      00000080H   SFRSYM    DATA     BYTE      P0
      000000C8H.1 SFRSYM    DATA     BIT       T2I1
      000000DFH   SFRSYM    DATA     BYTE      CCPDATO
      000000C5H   SFRSYM    DATA     BYTE      CCH2
      00000090H   SFRSYM    DATA     BYTE      P1
      000000C7H   SFRSYM    DATA     BYTE      CCH3
      000000A0H   SFRSYM    DATA     BYTE      P2
      00000098H.5 SFRSYM    DATA     BIT       SM20
      000000B0H   SFRSYM    DATA     BYTE      P3
      00000090H.2 SFRSYM    DATA     BIT       S1
      000000D0H.6 SFRSYM    DATA     BIT       AC
      000000C2H   SFRSYM    DATA     BYTE      CCL1
      00000090H.3 SFRSYM    DATA     BIT       S2
      000000C4H   SFRSYM    DATA     BYTE      CCL2
      00000090H.4 SFRSYM    DATA     BIT       S3
      000000D8H.7 SFRSYM    DATA     BIT       BD
      000000B8H   SFRSYM    DATA     BIT       RFSPI
      000000A8H.7 SFRSYM    DATA     BIT       EA
      000000CCH   SFRSYM    DATA     WORD      T2
      000000C6H   SFRSYM    DATA     BYTE      CCL3
      000000B7H   SFRSYM    DATA     BYTE      SPISRDSZ
      00000080H   SFRSYM    DATA     BIT       LED1
      00000080H.5 SFRSYM    DATA     BIT       LED2
      00000080H.1 SFRSYM    DATA     BIT       LED3
      000000C8H.3 SFRSYM    DATA     BIT       T2R0
      000000C8H.4 SFRSYM    DATA     BIT       T2R1
      000000A8H   SFRSYM    DATA     BYTE      IEN0
      000000B8H   SFRSYM    DATA     BYTE      IEN1
      000000A5H   SFRSYM    DATA     BYTE      WUCON
      00000085H   SFRSYM    DATA     BYTE      DPH1
      000000DBH   SFRSYM    DATA     BYTE      COMPCON
LX51 LINKER/LOCATER V4.17                                                             06/13/2011  13:18:25  PAGE 9


      000000A3H   SFRSYM    DATA     BYTE      CLKCTRL
      00000084H   SFRSYM    DATA     BYTE      DPL1
      000000C8H.5 SFRSYM    DATA     BIT       I2FR
      000000B8H.3 SFRSYM    DATA     BIT       WUPIN
      000000C8H.6 SFRSYM    DATA     BIT       I3FR
      000000FFH   SFRSYM    DATA     BYTE      SPIMDAT
      000000C0H.7 SFRSYM    DATA     BIT       EXF2
      00000098H.4 SFRSYM    DATA     BIT       REN0
      000000C8H.2 SFRSYM    DATA     BIT       T2CM
      000000B8H.1 SFRSYM    DATA     BIT       RF
      000000B8H.5 SFRSYM    DATA     BIT       WUIRQ
      000000E7H   SFRSYM    DATA     BYTE      SPIRDAT
      000000C1H   SFRSYM    DATA     BYTE      CCEN
      000000E2H   SFRSYM    DATA     BYTE      W2CON0
      000000BFH   SFRSYM    DATA     BYTE      SPISDAT
      000000D0H.7 SFRSYM    DATA     BIT       CY
      000000E1H   SFRSYM    DATA     BYTE      W2CON1
      000000FBH   SFRSYM    DATA     BYTE      FDCR
      000000E8H   SFRSYM    DATA     BIT       RFCE
      000000CBH   SFRSYM    DATA     BYTE      CRCH
      00000081H   SFRSYM    DATA     BYTE      SP
      000000D0H.2 SFRSYM    DATA     BIT       OV
      000000CAH   SFRSYM    DATA     BYTE      CRCL
      000000ADH   SFRSYM    DATA     BYTE      CLKLFCTRL
      000000B1H   SFRSYM    DATA     BYTE      RSTREAS
      000000C8H.7 SFRSYM    DATA     BIT       T2PS
      000000F9H   SFRSYM    DATA     BYTE      FPCR
      000000B8H.4 SFRSYM    DATA     BIT       MISC
      000000A1H   SFRSYM    DATA     BYTE      PWMDC0
      000000B4H   SFRSYM    DATA     BYTE      RTC2CMP0
      000000A2H   SFRSYM    DATA     BYTE      PWMDC1
      000000B5H   SFRSYM    DATA     BYTE      RTC2CMP1
      00000080H   SFRSYM    DATA     BIT       P00
      000000BAH   SFRSYM    DATA     BYTE      S0RELH
      00000090H   SFRSYM    DATA     BIT       P10
      00000080H.1 SFRSYM    DATA     BIT       P01
      00000087H   SFRSYM    DATA     BYTE      PCON
      000000A0H   SFRSYM    DATA     BIT       P20
      00000090H.1 SFRSYM    DATA     BIT       P11
      00000080H.2 SFRSYM    DATA     BIT       P02
      000000B0H   SFRSYM    DATA     BIT       P30
      000000A0H.1 SFRSYM    DATA     BIT       P21
      00000090H.2 SFRSYM    DATA     BIT       P12
      00000080H.3 SFRSYM    DATA     BIT       P03
      000000C0H.2 SFRSYM    DATA     BIT       SPIF
      000000F8H.2 SFRSYM    DATA     BIT       RDIS
      000000B0H.1 SFRSYM    DATA     BIT       P31
      000000A0H.2 SFRSYM    DATA     BIT       P22
      00000090H.3 SFRSYM    DATA     BIT       P13
      00000080H.4 SFRSYM    DATA     BIT       P04
      000000AAH   SFRSYM    DATA     BYTE      S0RELL
      000000B0H.2 SFRSYM    DATA     BIT       P32
      000000A0H.3 SFRSYM    DATA     BIT       P23
      00000090H.4 SFRSYM    DATA     BIT       P14
      00000080H.5 SFRSYM    DATA     BIT       P05
      000000D9H   SFRSYM    DATA     BYTE      W2SADR
      00000089H   SFRSYM    DATA     BYTE      TMOD
      00000088H   SFRSYM    DATA     BYTE      TCON
      000000B0H.3 SFRSYM    DATA     BIT       P33
      000000A0H.4 SFRSYM    DATA     BIT       P24
      00000090H.5 SFRSYM    DATA     BIT       P15
      00000080H.6 SFRSYM    DATA     BIT       P06
      000000B0H.4 SFRSYM    DATA     BIT       P34
      000000A0H.5 SFRSYM    DATA     BIT       P25
      00000090H.6 SFRSYM    DATA     BIT       P16
LX51 LINKER/LOCATER V4.17                                                             06/13/2011  13:18:25  PAGE 10


      00000080H.7 SFRSYM    DATA     BIT       P07
      000000C2H   SFRSYM    DATA     WORD      CC1
      000000B0H.5 SFRSYM    DATA     BIT       P35
      000000A0H.6 SFRSYM    DATA     BIT       P26
      00000090H.7 SFRSYM    DATA     BIT       P17
      000000C4H   SFRSYM    DATA     WORD      CC2
      000000B0H.6 SFRSYM    DATA     BIT       P36
      000000A0H.7 SFRSYM    DATA     BIT       P27
      000000C6H   SFRSYM    DATA     WORD      CC3
      000000B0H.7 SFRSYM    DATA     BIT       P37
      000000E8H.2 SFRSYM    DATA     BIT       RFCKEN
      000000F8H   SFRSYM    DATA     BIT       WPEN
      000000DDH   SFRSYM    DATA     BYTE      CCPDATIA
      000000DEH   SFRSYM    DATA     BYTE      CCPDATIB
      00000088H.1 SFRSYM    DATA     BIT       IE0
      000000F8H.4 SFRSYM    DATA     BIT       RDYN
      00000088H.3 SFRSYM    DATA     BIT       IE1
      000000CFH   SFRSYM    DATA     BYTE      WUOPC0
      000000F0H   SFRSYM    DATA     BYTE      B
      000000E9H   SFRSYM    DATA     BYTE      MD0
      000000CEH   SFRSYM    DATA     BYTE      WUOPC1
      000000A7H   SFRSYM    DATA     BYTE      MEMCON
      000000EAH   SFRSYM    DATA     BYTE      MD1
      000000D7H   SFRSYM    DATA     BYTE      RNGDAT
      000000EBH   SFRSYM    DATA     BYTE      MD2
      000000ECH   SFRSYM    DATA     BYTE      MD3
      000000EDH   SFRSYM    DATA     BYTE      MD4
      000000AFH   SFRSYM    DATA     BYTE      WDSV
      000000EEH   SFRSYM    DATA     BYTE      MD5
      000000E0H   SFRSYM    DATA     BYTE      ACC
      000000DCH   SFRSYM    DATA     BYTE      POFCON
      000000A8H.4 SFRSYM    DATA     BIT       ES0
      000000A8H.1 SFRSYM    DATA     BIT       ET0
      000000A9H   SFRSYM    DATA     BYTE      IP0
      000000A8H.3 SFRSYM    DATA     BIT       ET1
      00000088H.5 SFRSYM    DATA     BIT       TF0
      000000B9H   SFRSYM    DATA     BYTE      IP1
      000000A8H.5 SFRSYM    DATA     BIT       ET2
      00000098H   SFRSYM    DATA     BIT       RI0
      00000088H.7 SFRSYM    DATA     BIT       TF1
      000000C0H   SFRSYM    DATA     BIT       RFSPIF
      000000C0H.6 SFRSYM    DATA     BIT       TF2
      000000FCH   SFRSYM    DATA     BYTE      SPIMCON0
      000000D6H   SFRSYM    DATA     BYTE      RNGCTL
      0000008CH   SFRSYM    DATA     BYTE      TH0
      000000A8H   SFRSYM    DATA     BIT       EX0
      00000098H.1 SFRSYM    DATA     BIT       TI0
      00000088H   SFRSYM    DATA     BIT       IT0
      000000FDH   SFRSYM    DATA     BYTE      SPIMCON1
      0000008DH   SFRSYM    DATA     BYTE      TH1
      000000A8H.2 SFRSYM    DATA     BIT       EX1
      00000088H.2 SFRSYM    DATA     BIT       IT1
      000000CDH   SFRSYM    DATA     BYTE      TH2
      000000AEH   SFRSYM    DATA     BYTE      OPMCON
      000000D0H   SFRSYM    DATA     BIT       P
      00000098H.7 SFRSYM    DATA     BIT       SM0
      0000008AH   SFRSYM    DATA     BYTE      TL0
      00000098H.6 SFRSYM    DATA     BIT       SM1
      000000E4H   SFRSYM    DATA     BYTE      SPIRCON0
      0000008BH   SFRSYM    DATA     BYTE      TL1
      000000E5H   SFRSYM    DATA     BYTE      SPIRCON1
      000000CCH   SFRSYM    DATA     BYTE      TL2
      000000BCH   SFRSYM    DATA     BYTE      SPISCON0
      000000BDH   SFRSYM    DATA     BYTE      SPISCON1
      000000D0H.3 SFRSYM    DATA     BIT       RS0
LX51 LINKER/LOCATER V4.17                                                             06/13/2011  13:18:25  PAGE 11


      00000088H.4 SFRSYM    DATA     BIT       TR0
      000000D0H.4 SFRSYM    DATA     BIT       RS1
      000000B2H   SFRSYM    DATA     BYTE      PWMCON
      00000088H.6 SFRSYM    DATA     BIT       TR1
      000000CAH   SFRSYM    DATA     WORD      CRC
      000000A6H   SFRSYM    DATA     BYTE      INTEXP
      000000C0H.3 SFRSYM    DATA     BIT       WUPINF
      000000FAH   SFRSYM    DATA     BYTE      FCR
      000000D3H   SFRSYM    DATA     BYTE      ADCCON1
      000000D2H   SFRSYM    DATA     BYTE      ADCCON2
      00000083H   SFRSYM    DATA     BYTE      DPH
      000000D1H   SFRSYM    DATA     BYTE      ADCCON3
      000000C0H.1 SFRSYM    DATA     BIT       RFF
      00000093H   SFRSYM    DATA     BYTE      P0DIR
      00000082H   SFRSYM    DATA     BYTE      DPL
      0000009EH   SFRSYM    DATA     BYTE      P0CON
      00000099H   SFRSYM    DATA     BYTE      S0BUF
      00000094H   SFRSYM    DATA     BYTE      P1DIR
      0000009FH   SFRSYM    DATA     BYTE      P1CON
      00000095H   SFRSYM    DATA     BYTE      P2DIR
      000000B8H.7 SFRSYM    DATA     BIT       EXEN2
      000000DAH   SFRSYM    DATA     BYTE      W2DAT
      00000097H   SFRSYM    DATA     BYTE      P2CON
      00000096H   SFRSYM    DATA     BYTE      P3DIR
      000000A4H   SFRSYM    DATA     BYTE      PWRDWN
      00000098H   SFRSYM    DATA     BYTE      S0CON
      0000008FH   SFRSYM    DATA     BYTE      P3CON
      000000B6H   SFRSYM    DATA     BYTE      RTC2CPT00
      000000D8H   SFRSYM    DATA     BYTE      ADCON
      000000ACH   SFRSYM    DATA     BYTE      RTC2CPT10
      000000ABH   SFRSYM    DATA     BYTE      RTC2CPT01
      000000C8H   SFRSYM    DATA     BYTE      T2CON
      00000092H   SFRSYM    DATA     BYTE      DPS
      000000F8H.5 SFRSYM    DATA     BIT       WEN
      000000F8H   SFRSYM    DATA     BYTE      FSR
      000000D4H   SFRSYM    DATA     BYTE      ADCDATH
      000000C9H   SFRSYM    DATA     BYTE      MPAGE
      000000B8H.2 SFRSYM    DATA     BIT       SPI
      000000F8H.1 SFRSYM    DATA     BIT       RDEND
      000000D5H   SFRSYM    DATA     BYTE      ADCDATL
      000000F8H.3 SFRSYM    DATA     BIT       INFEN
      000000F8H.7 SFRSYM    DATA     BIT       MCDIS
      000000C0H.5 SFRSYM    DATA     BIT       WUF
      000000C0H.4 SFRSYM    DATA     BIT       MISCF
      000000EFH   SFRSYM    DATA     BYTE      ARCON
      000000D0H.5 SFRSYM    DATA     BIT       F0
      000000F8H.6 SFRSYM    DATA     BIT       STP
      000000FEH   SFRSYM    DATA     BYTE      SPIMSTAT
      000000E8H   SFRSYM    DATA     BYTE      RFCON
      000000D0H   SFRSYM    DATA     BYTE      PSW
      00000098H.2 SFRSYM    DATA     BIT       RB80
      000000C0H   SFRSYM    DATA     BYTE      IRCON
      000000E8H.1 SFRSYM    DATA     BIT       RFCSN
      000000E6H   SFRSYM    DATA     BYTE      SPIRSTAT
      000000B3H   SFRSYM    DATA     BYTE      RTC2CON

      010001BEH   BLOCK     CODE     ---       LVL=0
      00000006H   SYMBOL    DATA     WORD      x
      010001BEH   BLOCK     CODE     NEAR LAB  LVL=1
      00000004H   SYMBOL    DATA     WORD      i
      02000001H   SYMBOL    PDATA    WORD      j
      ---         BLOCKEND  ---      ---       LVL=1
      010001BEH   LINE      CODE     ---       #75
      010001BEH   LINE      CODE     ---       #76
      010001BEH   LINE      CODE     ---       #78
LX51 LINKER/LOCATER V4.17                                                             06/13/2011  13:18:25  PAGE 12


      010001C1H   LINE      CODE     ---       #79
      010001C8H   LINE      CODE     ---       #80
      010001C8H   LINE      CODE     ---       #81
      010001D0H   LINE      CODE     ---       #83
      010001E2H   LINE      CODE     ---       #84
      010001E9H   LINE      CODE     ---       #85
      ---         BLOCKEND  ---      ---       LVL=0

      01000284H   BLOCK     CODE     ---       LVL=0
      00000007H   SYMBOL    DATA     BYTE      value
      01000284H   LINE      CODE     ---       #89
      01000284H   LINE      CODE     ---       #90
      01000284H   LINE      CODE     ---       #91
      01000286H   LINE      CODE     ---       #93
      0100028BH   LINE      CODE     ---       #95
      0100028DH   LINE      CODE     ---       #96
      ---         BLOCKEND  ---      ---       LVL=0

      0100023DH   BLOCK     CODE     ---       LVL=0
      00000007H   SYMBOL    DATA     BYTE      reg
      00000005H   SYMBOL    DATA     BYTE      value
      0100023DH   BLOCK     CODE     NEAR LAB  LVL=1
      00000006H   SYMBOL    DATA     BYTE      status
      ---         BLOCKEND  ---      ---       LVL=1
      0100023DH   LINE      CODE     ---       #100
      0100023DH   LINE      CODE     ---       #101
      0100023DH   LINE      CODE     ---       #104
      0100023FH   LINE      CODE     ---       #105
      01000244H   LINE      CODE     ---       #106
      01000249H   LINE      CODE     ---       #107
      0100024BH   LINE      CODE     ---       #109
      0100024DH   LINE      CODE     ---       #110
      ---         BLOCKEND  ---      ---       LVL=0

      0100025DH   BLOCK     CODE     ---       LVL=0
      00000007H   SYMBOL    DATA     BYTE      reg
      0100025DH   BLOCK     CODE     NEAR LAB  LVL=1
      00000007H   SYMBOL    DATA     BYTE      reg_val
      ---         BLOCKEND  ---      ---       LVL=1
      0100025DH   LINE      CODE     ---       #114
      0100025DH   LINE      CODE     ---       #115
      0100025DH   LINE      CODE     ---       #118
      0100025FH   LINE      CODE     ---       #119
      01000262H   LINE      CODE     ---       #120
      01000267H   LINE      CODE     ---       #121
      01000269H   LINE      CODE     ---       #123
      01000269H   LINE      CODE     ---       #124
      ---         BLOCKEND  ---      ---       LVL=0

      0100000EH   BLOCK     CODE     ---       LVL=0
      00000007H   SYMBOL    DATA     BYTE      reg
      02000002H   SYMBOL    PDATA    ---       pBuf
      02000005H   SYMBOL    PDATA    BYTE      bytes
      01000018H   BLOCK     CODE     NEAR LAB  LVL=1
      00000006H   SYMBOL    DATA     BYTE      status
      00000005H   SYMBOL    DATA     BYTE      byte_ctr
      ---         BLOCKEND  ---      ---       LVL=1
      0100000EH   LINE      CODE     ---       #128
      01000018H   LINE      CODE     ---       #129
      01000018H   LINE      CODE     ---       #132
      0100001AH   LINE      CODE     ---       #133
      0100001FH   LINE      CODE     ---       #134
      0100002AH   LINE      CODE     ---       #135
      01000045H   LINE      CODE     ---       #136
      01000047H   LINE      CODE     ---       #137
LX51 LINKER/LOCATER V4.17                                                             06/13/2011  13:18:25  PAGE 13


      01000049H   LINE      CODE     ---       #138
      ---         BLOCKEND  ---      ---       LVL=0

      01000298H   BLOCK     CODE     ---       LVL=0
      01000298H   LINE      CODE     ---       #142
      01000298H   LINE      CODE     ---       #143
      01000298H   LINE      CODE     ---       #144
      0100029AH   LINE      CODE     ---       #145
      ---         BLOCKEND  ---      ---       LVL=0

      0100014FH   BLOCK     CODE     ---       LVL=0
      0100014FH   LINE      CODE     ---       #150
      0100014FH   LINE      CODE     ---       #151
      0100014FH   LINE      CODE     ---       #152
      01000156H   LINE      CODE     ---       #153
      01000159H   LINE      CODE     ---       #154
      0100015CH   LINE      CODE     ---       #155
      0100015FH   LINE      CODE     ---       #158
      01000162H   LINE      CODE     ---       #159
      01000165H   LINE      CODE     ---       #160
      01000168H   LINE      CODE     ---       #161
      0100016BH   LINE      CODE     ---       #162
      0100016EH   LINE      CODE     ---       #163
      0100017DH   LINE      CODE     ---       #164
      0100017FH   LINE      CODE     ---       #165
      01000186H   LINE      CODE     ---       #166
      01000188H   LINE      CODE     ---       #167
      ---         BLOCKEND  ---      ---       LVL=0

      010000FAH   BLOCK     CODE     ---       LVL=0
      010000FAH   LINE      CODE     ---       #171
      010000FAH   LINE      CODE     ---       #172
      010000FAH   LINE      CODE     ---       #173
      010000FCH   LINE      CODE     ---       #174
      010000FEH   LINE      CODE     ---       #175
      01000100H   LINE      CODE     ---       #177
      01000107H   LINE      CODE     ---       #179
      01000117H   LINE      CODE     ---       #180
      01000127H   LINE      CODE     ---       #182
      0100012EH   LINE      CODE     ---       #183
      01000133H   LINE      CODE     ---       #184
      0100013AH   LINE      CODE     ---       #185
      01000141H   LINE      CODE     ---       #186
      01000148H   LINE      CODE     ---       #187
      ---         BLOCKEND  ---      ---       LVL=0

      010001EAH   BLOCK     CODE     ---       LVL=0
      010001EAH   LINE      CODE     ---       #192
      010001F7H   LINE      CODE     ---       #194
      010001FEH   LINE      CODE     ---       #195
      01000205H   LINE      CODE     ---       #196
      ---         BLOCKEND  ---      ---       LVL=0

      0100024EH   BLOCK     CODE     ---       LVL=0
      0100024EH   LINE      CODE     ---       #201
      0100024EH   LINE      CODE     ---       #202
      0100024EH   LINE      CODE     ---       #203
      01000251H   LINE      CODE     ---       #204
      01000254H   LINE      CODE     ---       #205
      01000257H   LINE      CODE     ---       #206
      0100025AH   LINE      CODE     ---       #207
      0100025CH   LINE      CODE     ---       #208
      ---         BLOCKEND  ---      ---       LVL=0

      0100026AH   BLOCK     CODE     ---       LVL=0
LX51 LINKER/LOCATER V4.17                                                             06/13/2011  13:18:25  PAGE 14


      0100026AH   LINE      CODE     ---       #213
      0100026AH   LINE      CODE     ---       #214
      0100026AH   LINE      CODE     ---       #215
      0100026CH   LINE      CODE     ---       #216
      0100026FH   LINE      CODE     ---       #217
      01000271H   LINE      CODE     ---       #218
      01000274H   LINE      CODE     ---       #219
      01000276H   LINE      CODE     ---       #222
      ---         BLOCKEND  ---      ---       LVL=0

      010002A9H   BLOCK     CODE     ---       LVL=0
      010002A9H   LINE      CODE     ---       #228
      010002A9H   LINE      CODE     ---       #229
      010002A9H   LINE      CODE     ---       #230
      010002ACH   LINE      CODE     ---       #231
      ---         BLOCKEND  ---      ---       LVL=0

      010002ADH   BLOCK     CODE     ---       LVL=0
      010002ADH   LINE      CODE     ---       #235
      010002ADH   LINE      CODE     ---       #236
      010002ADH   LINE      CODE     ---       #237
      010002B0H   LINE      CODE     ---       #238
      ---         BLOCKEND  ---      ---       LVL=0

      01000068H   BLOCK     CODE     ---       LVL=0
      01000068H   LINE      CODE     ---       #242
      01000068H   LINE      CODE     ---       #244
      0100006AH   LINE      CODE     ---       #245
      ---         BLOCKEND  ---      ---       LVL=0

      01000277H   BLOCK     CODE     ---       LVL=0
      01000277H   LINE      CODE     ---       #250
      01000277H   LINE      CODE     ---       #253
      01000279H   LINE      CODE     ---       #254
      0100027CH   LINE      CODE     ---       #255
      0100027FH   LINE      CODE     ---       #256
      01000281H   LINE      CODE     ---       #257
      01000283H   LINE      CODE     ---       #258
      ---         BLOCKEND  ---      ---       LVL=0

      0100004EH   BLOCK     CODE     ---       LVL=0
      0100004EH   LINE      CODE     ---       #262
      0100004EH   LINE      CODE     ---       #263
      0100004EH   LINE      CODE     ---       #264
      01000051H   LINE      CODE     ---       #265
      01000054H   LINE      CODE     ---       #267
      0100005AH   LINE      CODE     ---       #268
      01000061H   LINE      CODE     ---       #269
      01000067H   LINE      CODE     ---       #270
      ---         BLOCKEND  ---      ---       LVL=0

      0100028EH   BLOCK     CODE     ---       LVL=0
      0100028EH   LINE      CODE     ---       #274
      0100028EH   LINE      CODE     ---       #275
      0100028EH   LINE      CODE     ---       #276
      01000291H   LINE      CODE     ---       #277
      01000294H   LINE      CODE     ---       #278
      01000297H   LINE      CODE     ---       #279
      ---         BLOCKEND  ---      ---       LVL=0

      01000003H   BLOCK     CODE     ---       LVL=0
      01000003H   BLOCK     CODE     NEAR LAB  LVL=1
      00000007H   SYMBOL    DATA     BYTE      temp
      ---         BLOCKEND  ---      ---       LVL=1
      01000003H   LINE      CODE     ---       #284
LX51 LINKER/LOCATER V4.17                                                             06/13/2011  13:18:25  PAGE 15


      01000003H   LINE      CODE     ---       #285
      01000003H   LINE      CODE     ---       #287
      01000005H   LINE      CODE     ---       #288
      01000008H   LINE      CODE     ---       #289
      0100000AH   LINE      CODE     ---       #291
      ---         BLOCKEND  ---      ---       LVL=0

      010002A1H   BLOCK     CODE     ---       LVL=0
      010002A1H   BLOCK     CODE     NEAR LAB  LVL=1
      00000007H   SYMBOL    DATA     BYTE      value
      ---         BLOCKEND  ---      ---       LVL=1
      010002A1H   LINE      CODE     ---       #296
      010002A1H   LINE      CODE     ---       #297
      010002A1H   LINE      CODE     ---       #299
      010002A6H   LINE      CODE     ---       #301
      010002A8H   LINE      CODE     ---       #302
      010002A8H   LINE      CODE     ---       #303
      ---         BLOCKEND  ---      ---       LVL=0

      01000189H   BLOCK     CODE     ---       LVL=0
      01000189H   BLOCK     CODE     NEAR LAB  LVL=1
      00000007H   SYMBOL    DATA     BYTE      del_val_high
      02000000H   SYMBOL    PDATA    BYTE      del_val_low
      ---         BLOCKEND  ---      ---       LVL=1
      01000189H   LINE      CODE     ---       #308
      01000189H   LINE      CODE     ---       #309
      01000189H   LINE      CODE     ---       #312
      0100018CH   LINE      CODE     ---       #313
      0100018FH   LINE      CODE     ---       #316
      01000191H   LINE      CODE     ---       #318
      01000194H   LINE      CODE     ---       #322
      01000194H   LINE      CODE     ---       #323
      01000194H   LINE      CODE     ---       #324
      01000197H   LINE      CODE     ---       #325
      0100019AH   LINE      CODE     ---       #326
      0100019DH   LINE      CODE     ---       #327
      0100019FH   LINE      CODE     ---       #329
      010001A2H   LINE      CODE     ---       #330
      010001A5H   LINE      CODE     ---       #331
      010001A8H   LINE      CODE     ---       #332
      010001AAH   LINE      CODE     ---       #337
      010001ADH   LINE      CODE     ---       #338
      010001B3H   LINE      CODE     ---       #339
      010001B6H   LINE      CODE     ---       #341
      010001BCH   LINE      CODE     ---       #345
      ---         BLOCKEND  ---      ---       LVL=0

      ---         MODULE    ---      ---       ?C_INIT
      010000B5H   PUBLIC    CODE     ---       ?C_START

      ---         MODULE    ---      ---       ?C?CLDPTR
      01000210H   PUBLIC    CODE     ---       ?C?CLDPTR



*** WARNING L16: UNCALLED FUNCTION, IGNORED FOR OVERLAY PROCESS
    NAME:    PD_MODE/MAIN

*** WARNING L16: UNCALLED FUNCTION, IGNORED FOR OVERLAY PROCESS
    NAME:    RTC2_INIT/MAIN

*** WARNING L16: UNCALLED FUNCTION, IGNORED FOR OVERLAY PROCESS
    NAME:    RTC0_INIT/MAIN

*** WARNING L16: UNCALLED FUNCTION, IGNORED FOR OVERLAY PROCESS
LX51 LINKER/LOCATER V4.17                                                             06/13/2011  13:18:25  PAGE 16


    NAME:    RTC2_ON/MAIN

*** WARNING L16: UNCALLED FUNCTION, IGNORED FOR OVERLAY PROCESS
    NAME:    RTC2_OFF/MAIN

Program Size: data=20.0 xdata=11 const=0 code=688
LX51 RUN COMPLETE.  5 WARNING(S),  0 ERROR(S)
